:020000040000FA
:0400000027EF02F0F4
:040008000EEF00F007
:0800180040EF00F09EA221EF71
:1000200000F09E92A52BA5B1110000EE80F010EE1D
:1000300092F0080EA46FFF0ED76EFF0ED66ED58E0F
:100040001100E61C8116E61C8216D59EF294A407C8
:10005000EE1CD76EEE1CD66EA453D8A4D58E00002D
:100060000000000000000000000000000000000090
:10007000000000000000E6508112E55082121100DD
:100080001000A69CA69EA19865C0A8FF64C0A9FF09
:10009000A684550EA76EAA0EA76EA682A1A84EEF43
:1000A00000F0A6941200A69CA69E64C0A9FFA6809C
:1000B000A8CF65F01200080E616F62AF829A62BF2E
:1000C000828A0000808A809A6237612F5DEF00F09B
:1000D0001200948A080E616F626BD890623782BA00
:1000E0006281808A809A612F6EEF00F0949A1200EC
:1000F0008098450E626F5BEC00F069EC00F062C026
:10010000A6F069EC00F062C068F069EC00F062C033
:1001100069F069EC00F062C06AF069EC00F062C05E
:100120006BF069EC00F062C071F069EC00F062C045
:1001300070F069EC00F062C073F069EC00F062C02E
:1001400072F069EC00F062C075F069EC00F062C01A
:1001500074F069EC00F062C077F069EC00F062C006
:1001600076F069EC00F062C079F069EC00F062C0F2
:1001700078F069EC00F062C07BF069EC00F062C0DE
:100180007AF069EC00F062C07DF069EC00F062C0CA
:100190007CF069EC00F062C07FF069EC00F062C0B6
:1001A0007EF0808812008098000E626F5BEC00F099
:1001B000000E626F5BEC00F080888098060E626F24
:1001C0005BEC00F0540E626F5BEC00F0750E626F3A
:1001D0005BEC00F0C50E626F5BEC00F02A0E626F04
:1001E0005BEC00F080888098460E626F5BEC00F05C
:1001F00069EC00F062C068F069EC00F062C069F080
:1002000069EC00F062C06AF069EC00F062C06BF06B
:100210008088060EF76E940EF66EFF0E636F330E37
:10022000606F632B0900F528FCE0809863C062F0E2
:100230005BEC00F0F5CF62F05BEC00F08088602FA3
:1002400011EF01F08098020E626F5BEC00F0010E7E
:10025000626F5BEC00F080888098020E626F628DA6
:100260005BEC00F0000069EC00F0808862B12CEFDC
:1002700001F08098240E626F5BEC00F0130E626F49
:100280005BEC00F080888098260E626F5BEC00F0DB
:100290003B0E626F5BEC00F0808880980F0E626FFF
:1002A0005BEC00F0000E626F5BEC00F080888098E1
:1002B000020E626F5BEC00F0020E626F5BEC00F00E
:1002C00080888098020E626F628D5BEC00F0000007
:1002D00069EC00F0808862B361EF01F080980F0E46
:1002E000626F5BEC00F0A00E626F5BEC00F0808848
:1002F0008098020E626F5BEC00F0020E626F5BECA6
:1003000000F080888098020E626F628D5BEC00F0D6
:10031000000069EC00F0808862B382EF01F0809801
:10032000250E626F5BEC00F0080E626F5BEC00F074
:1003300080881200676B8098A00E626F5BEC00F003
:1003400080888098F00E626F5BEC00F08088809867
:100350000F0E626F5BEC00F0000E626F5BEC00F062
:1003600080888098C00E626F5BEC00F08088B1904E
:10037000270EB36EB31E100EB26EB21EA192B180E4
:10038000A1A2C0EF01F067B5829C67A5828C82A014
:10039000CFEF01F0672FB7EF01F0FEEF01F080988B
:1003A000000E626F628D5BEC00F0000069EC00F003
:1003B000808862BB9BEF01F062BD9BEF01F078EC9F
:1003C00000F0646B68C065F041EC00F0642B69C01C
:1003D00065F041EC00F0642B6AC065F041EC00F080
:1003E000642B6BC065F041EC00F068C06CF069C034
:1003F0006DF06AC06EF06BC06FF01200646B53EC6E
:1004000000F065C06CF0642B53EC00F065C06DF03B
:10041000642B53EC00F065C06EF0642B53EC00F0DD
:1004200065C06FF01200902F20EF02F0100E906F59
:10043000060EF76EC80EF66E9151F626D8B0F72A62
:100440000900F504666F6C390F0B665F1200D38CE0
:10045000D38AD388806A816A826A828C949C8088DD
:100460009298828A949A809A929A939C939A93985B
:10047000949494929496939E949E7E6A7F6A000EC2
:10048000926F000E936F400E946F000E956F200ECA
:10049000966F000E976F100E986F000E996F000EFA
:1004A0009A6F040E9B6F000E9C6F020E9D6F000EE4
:1004B0009E6F080E9F6F800EA06F000EA16F000E42
:1004C000A26F800EA36FD56AD580F294F28AF90EDE
:1004D000CB6ECA6ACA8CCA86CA829E929D829F824D
:1004E000F28CF28EB16AB18EB18AA192DC0E816F6C
:1004F000836F856F876F896F8B6F8D6F8F6F050E21
:10050000806F826F846F866F886F8A6F8C6F8E6F3B
:10051000CA84B190270EB36EB31E100EB26EB21E17
:10052000A192B180A1A292EF02F0D3EC00F0000002
:100530009AEC01F08098460E626F5BEC00F069EC7B
:1005400000F0620E686F69EC00F0620E696F69EC92
:1005500000F0620E6A6F69EC00F0620E6B6F8088CB
:100560006C39F00B916F010E906F13EC02F08098D4
:10057000A00E626F5BEC00F080888098F00E626FD6
:100580005BEC00F0808880980F0E626F5BEC00F0EF
:1005900066C062F05BEC00F080888098C00E626FED
:1005A0005BEC00F08088B190070EB36EB31ED00EE6
:1005B000B26EB21EA192B180A1B245EF03F082B03B
:1005C000DCEF02F08098000E626F628D5BEC00F051
:1005D000000069EC00F0808862BBDCEF02F062BDD5
:1005E000DCEF02F078EC00F06C516863DCEF02F0B5
:1005F0006D516963DCEF02F06E516A63DCEF02F06B
:100600006F516B63DCEF02F0828CF29E70C080F061
:1006100071C081F0F28E00000000F29E72C082F084
:1006200073C083F0F28E00000000F29E74C084F06C
:1006300075C085F0F28E00000000F29E76C086F054
:1006400077C087F0F28E00000000F29E78C088F03C
:1006500079C089F0F28E00000000F29E7AC08AF024
:100660007BC08BF0F28E00000000F29E7CC08CF00C
:100670007DC08DF0F28E00000000F29E7EC08EF0F4
:100680007FC08FF0F28EB5EF02F0829C13EC02F087
:10069000B5EF02F0FF42001400FFFF000000000170
:1006A000210500509E4B0002162B12006280800034
:1006B0000A32C30F13C300FF00003B00174780033B
:1006C00001451800010FFF000A5A14641E6E2878B5
:1006D00032823C8C469650A0A05096468C3C82328A
:1006E00078286E1E64145A0A0A5A50A0146446965A
:1006F0001E6E3C8C28783282823278288C3C6E1EAA
:1007000096466414A0505A0A28780A5A50A01464D5
:100710001E6E3C8C32824696964682328C3C6E1E11
:100720006414A0505A0A782850A028780A5A1E6EDD
:100730003C8C3282469614646414964682328C3C19
:100740006E1E5A0A7828A05050A046963C8C2878F5
:100750000A5A32821E6E146464146E1E82325A0A61
:1007600078288C3C9646A05046963C8C50A0287821
:100770000A5A1E6E32821464641482326E1E5A0A41
:100780007828A0508C3C964646960A5A3C8C1464B5
:1007900050A028781E6E328282326E1E7828A050B9
:1007A00064148C3C5A0A964646960A5A50A03C8CD1
:1007B00028781E6E32821464641482326E1E782889
:0807C0008C3CA0505A0A964639
:020000040030CA
:0400000000082914B7
:02000500800079
:0600080003C003E0034009
:0200000400F00A
:040000004D434850D4
:00000001FF
